:1000000012C02AC029C028C027C026C025C024C0CD
:1000100023C022C021C020C01FC01EC01DC01CC0E4
:100020001BC01AC019C011241FBECFEDCDBF10E0F8
:10003000A0E6B0E0E2E2F2E002C005900D92A03648
:10004000B107D9F710E0A0E6B0E001C01D92A236DA
:10005000B107E1F75DD0E3C0D3CF86B3E0E2FEE4C1
:100060003197F1F736B390E080729070959587954F
:100070009595879595958795959587959595879568
:10008000882319F420E0822F089520E0832F90E048
:10009000807290709595879595958795959587959C
:1000A0009595879595958795882321F081E0282758
:1000B000822F089521E081E02827FACF8091600007
:1000C0008F5F80936000843040F010926000C39A8C
:1000D000C49AC09AC198C2980895813039F081308D
:1000E000B0F3823079F0833039F00895C398C49A20
:1000F000C098C19AC2980895C398C498C09AC198EC
:10010000C29A0895C39AC498C098C198C29A089593
:100110000F931F93CF93DF938FED87BB10926000F7
:10012000C39AC09AC198C2981092610000E21EE47E
:10013000C8ECD0E03091610086B3F8013197F1F757
:1001400026B390E0807290709595879595958795E8
:10015000959587959595879595958795882309F425
:1001600054C0822F90E080729070959587959595F8
:1001700087959595879595958795959587958823E6
:1001800009F443C0332309F040C020E23EE4CE012D
:100190000197F1F721503040D1F731E086B3F801F3
:1001A0003197F1F726B390E080729070959587951E
:1001B0009595879595958795959587959595879527
:1001C000882309F4B9CF822F90E0807290709595C2
:1001D0008795959587959595879595958795959507
:1001E0008795882309F4A8CF332309F4A5CF30934A
:1001F000610064DF1092610028EE33E0CE010197C8
:10020000F1F721503040D1F795CF28EE33E0CE0101
:100210000197F1F721503040D1F730E0BFCFF8948B
:02022000FFCF0E
:00000001FF
